:020000040800F2
:100000003808002089010008F52200085D2000085A
:10001000F122000861020008192700080000000012
:10002000000000000000000000000000FD220008A9
:100030007D02000800000000F922000801230008EA
:10004000A3010008A3010008A3010008A301000800
:10005000A3010008A3010008A3010008A3010008F0
:10006000A3010008A3010008A3010008A3010008E0
:10007000A3010008A3010008A3010008A3010008D0
:100080006502000871020008A3010008A30100082E
:10009000A3010008A3010008A3010008A3010008B0
:1000A000A3010008A3010008A3010008A3010008A0
:1000B000A3010008A3010008A3010008A301000890
:1000C000A3010008A3010008A3010008A301000880
:1000D000A3010008A30100080D270008A3010008E0
:1000E000A3010008A3010008A301000800F002F822
:1000F00000F03AF80AA090E8000C82448344AAF188
:100100000107DA4501D100F02FF8AFF2090EBAE885
:100110000F0013F0010F18BFFB1A43F0010318473B
:100120000C4500002C450000103A24BF78C878C167
:10013000FAD8520724BF30C830C144BF04680C60ED
:10014000704700000023002400250026103A28BF35
:1001500078C1FBD8520728BF30C148BF0B60704739
:100160001FB51FBD10B510BD00F044F81146FFF7D4
:10017000F7FF02F07BFB00F062F803B4FFF7F2FF39
:1001800003BC00F065F800000948804709480047B3
:10019000FEE7FEE7FEE7FEE7FEE7FEE7FEE7FEE737
:1001A000FEE7FEE704480549054A064B7047000094
:1001B00005230008ED000008380200203808002060
:1001C000380400203804002070477047704710B58D
:1001D00000F008F8006810BD10B5044600F002F801
:1001E000046010BD004870471000002000487047B0
:1001F000100000207546FFF7F9FFAE46050069467E
:10020000534620F00700854618B020B5FFF7CAFF17
:10021000BDE820404FF000064FF000074FF0000807
:100220004FF0000BAC46ACE8C009ACE8C009ACE844
:10023000C009ACE8C00921F007018D46704710B530
:100240000446AFF300802046BDE81040FFF795BF9D
:1002500001491820ABBEFEE72600020070470000EF
:10026000FEE7000040F2D400C2F2000000F08EB8B9
:1002700040F21810C2F2000000F088B87047000089
:10028000EFF3108072B600BFFEE70000014690F861
:100290002100022816D10868D1E90FC3026822F0B4
:1002A0000E020260026822F001020260012000FAE0
:1002B00003F2CCF8042081F821000020002281F80C
:1002C00020207047042088630120002281F820202C
:1002D0007047000080B590F82110022924D10268EF
:1002E000116821F00E0111602F211368C4F2020180
:1002F0008A4240F20401C4F2020123F001031360B8
:1003000018DD3023C4F202039A421FD04423C4F202
:1003100002039A421ED05823C4F202039A421FD10C
:100320004FF4803324E000BF04218163012108469B
:1003300080BD00BF0823C4F202039A420ED01C23E2
:10034000C4F202039A420BD1102311E04FF48073E0
:100350000EE000BF4FF480530AE000BF012307E026
:1003600001F1680C4FF08073624508BF4FF48013B1
:100370000B60012180F82110426B002180F82010D1
:100380000AB190470021084680BD000010B5016801
:10039000D0E90FCEDCF800200B685C072CD50424D4
:1003A00004FA0EF4144027D00A68920603D40A68AF
:1003B00022F004020A602F22C4F20202914240F2AB
:1003C0000402C4F2020261DD3023C4F20203994246
:1003D00078D04423C4F20203994279D05823C4F25E
:1003E0000203994240F080804FF480231360C16A79
:1003F000002940F08480A1E09C0729D5022404FA5A
:100400000EF4144024D00A68920606D40A6822F03A
:100410000A020A60012280F821202F22C4F202027F
:10042000914240F20402C4F202023FDD3023C4F2E2
:100430000203994266D04423C4F20203994265D074
:100440005823C4F20203994266D14FF400336BE0A3
:100450001B0773D5082303FA0EF31A4008BF10BD1B
:100460000A6822F00E020A60012101FA0EF2CCF8AD
:100470000420816380F82110016B0022002980F89C
:1004800020205BD0BDE81040084700BF0823C4F21D
:100490000203994222D01C23C4F20203994223D1C1
:1004A00040231360C16A51BB48E000BF0823C4F277
:1004B000020399422ED01C23C4F2020399422BD18D
:1004C000202331E04FF480631360C16AB9B935E08D
:1004D0004FF480431360C16A89B92FE0042313608D
:1004E000C16A61B92AE000BF02F168044FF080637D
:1004F000A14208BF4FF480031360C16AF1B1BDE8A7
:10050000104008474FF400730EE000BF4FF4005353
:100510000AE000BF022307E002F168044FF0007315
:10052000A14208BF4FF400131360816A002280F8D3
:10053000202019B1BDE81040084700BF10BD0000E1
:10054000014600284FF0010008BF70472DE9F04335
:10055000D1F800C04FF6F873CBF6FD734CF6CD42E0
:100560006344CCF6CC42A3FB02236FF0030707EAF7
:1005700093030027C4F2020701F10C09C1E90F73CC
:100580000223D1E9012E99E87002D1F81C8081F88C
:100590002130DCF8003043F6F077BB431A4342EADF
:1005A0000E0222432A43324342EA090242EA080287
:1005B000CCF8002000228A6381F8210081F82020F5
:1005C0000020BDE8F0437047F0B590F820C0BCF1C2
:1005D000010F32D04FF0010E80F820E090F821C0DA
:1005E000BCF1010F26D14FF0020C80F821C04FF072
:1005F000000CC0F838C0D0E900C4C56AC66BDCF88E
:100600000070102C27F00107CCF80070006C0EFA77
:1006100000F070600846CCF8043004BF10460A466B
:10062000CCF80800CCF80C20DCF8000045B140F014
:100630000E000DE0002180F820100220F0BD00BF68
:1006400020F00400CCF80000DCF8000040F00A00C4
:10065000CCF80000DCF8000040F00100CCF800000D
:100660000020F0BDB0B5044600F020F9054640F288
:100670000000C2F200000078611C18BF044400BFF3
:1006800000F014F9401BA042FAD3B0BD2DE9F04FA1
:1006900082B00E68002E00F0FF8041F20042C4F2EA
:1006A0000102042340F2004E904208BF03234FF69C
:1006B000FF7CC4F2010E009300240123C1F2100C50
:1006C0004FF0000A4FF0000947E000BF012504F099
:1006D0000C030F279F402BEA070705FA03F33B4360
:1006E00042F82630D1F804B040F20C455FEACB2244
:1006F000DEF8082054BF22EA080242EA0802C4F2E7
:100700000105CEF808202A685FEA8B2354BF22EA4D
:10071000080242EA08022A605FEA8B33DEF804200E
:1007200054BF22EA080242EA08025FEACB33CEF85D
:100730000420DEF800204FF0010354BF22EA080233
:1007400042EA0802CEF800200E680AF1010A36FAE1
:100750000AF204F1040400F09F8003FA0AF816EA92
:10076000080FF1D04A68624512DC122A56D8DFE839
:1007700002F0350B45495555555555555555555567
:100780005555554D510000BFD1F80C9046E000BFC3
:100790004FF6FF75C1F22105AA420FDC0025C1F218
:1007A0001105AA421AD00025C1F21205AA4215D09D
:1007B0000025C1F22105AA4210D02FE00025C1F288
:1007C0002205AA420AD00025C1F23105AA4205D06D
:1007D0000025C1F23205AA4220D100BF8A684AB181
:1007E000012A14BFC0F81480C0F810804FF0080927
:1007F00014E000BF4FF0040910E000BFCA6802F126
:1008000008090BE04FF0000908E000BFCA6802F1D8
:10081000040903E0CA6802F10C0900BF224605463C
:10082000BAF1080F24BF203A04352E680F279740ED
:10083000BE4309FA02F232432A60CA79D2067FF532
:1008400083AF41F21803C4F202031A684FEA9A0612
:1008500042F001021A601A6840F6000302F0010239
:100860000192019AAEF57E7252F826B0C4F20103ED
:1008700098420FD040F60043C4F2010398423FF47F
:1008800025AF41F20003C4F20103009D984208BF66
:1008900002251CE700251AE702B0BDE8F08F000032
:1008A000002A08BF090401617047000040F23420AB
:1008B000C2F200000068704740F2000040F23421AC
:1008C000C2F20000C2F2000100780A681044086019
:1008D0007047000080B542F20000C4F202000168D7
:1008E00041F010010160032000F08AF80F2000F0B1
:1008F00005F800F027F8002080BD000070B540F238
:100900000006C2F2000640F208013278C2F200018D
:100910004FF47A730968B3FBF2F20446B1FBF2F1CB
:10092000084600F05FFB0F2C4FF0010508D838B9DE
:100930004FF0FF3021460022002500F035F87460AA
:10094000284670BD82B041F21800C4F2020001686E
:10095000022241F001010160016801F001010191F1
:100960000199416841F080514160406800F0805039
:10097000009000980420C4F20100016862F31A613B
:10098000016002B070470000002848BF704700F0C7
:100990001F01012202FA01F14EF200124009CEF2CB
:1009A000000242F82010704710B54EF60C5CCEF2F3
:1009B000000CDCF80030C3F3022E8EF00704042C88
:1009C00028BF0424BEF103034FF0FF3E0EFA04F4E7
:1009D00038BF0023A14399400EFA03F39A4300F075
:1009E0000F03043B1143634409010C3300F16042DF
:1009F000B0F1FF3FC8BF02F56443197010BD00009D
:100A00004EF60C51CEF200010A684FF6FF031A4071
:100A100060F30A2242F0806040F0FD700860704789
:100A20002DE9F04381B0002800F0858042F20008F3
:100A3000C4F202080446D8F800000D4600F0070092
:100A400088420CD2D8F8000020F007002843C8F8EC
:100A50000000D8F8000000F00700A8426BD1206821
:100A600041F204098107C4F2020917D5410705D5EF
:100A7000D9F8001041F4E061C9F80010010705D56C
:100A8000D9F8001041F46051C9F80010D9F80010ED
:100A9000A26821F0F0011143C9F80010C00741D14C
:100AA000D8F8000000F00700A8420CD9D8F80000E0
:100AB00020F007002843C8F80000D8F8000000F034
:100AC0000700A84237D12068410707D5D9F80010A0
:100AD000E26821F4E0611143C9F80010000708D56D
:100AE000D9F80000216920F4605040EAC100C9F83B
:100AF0000000D9F8002002F00C00082841F2002084
:100B0000C0F27A0050D144F21A63C2F38341C0F6B6
:100B10000003595CD2033BD440F60010C0F23D0004
:100B2000484341E0606802280AD001282AD159F8D8
:100B3000041C890308D4012001B0BDE8F08300BF84
:100B400059F8041C8901F6D5D9F8001021F00301E9
:100B50000843C9F80000FFF7A9FE064641F28837AE
:100B6000D9F80000616800F00C00B0EB810F97D05D
:100B7000FFF79CFE801BB842F2D9032001B0BDE80C
:100B8000F08300BF59F8041C8907D4D5DCE700BF07
:100B9000D9F8002044F21863C2F34042C0F60003C3
:100BA0009A5C4843B0FBF2F0D9F8001044F20062BE
:100BB000C1F30311C0F60002515C40F2080220FAB2
:100BC00001F140F20400C2F200000068C2F200022B
:100BD0001160FFF793FE002001B0BDE8F083000034
:100BE00040F2080041F20401C2F20000C4F2020126
:100BF0000068096844F21062C1F30221C0F60002E5
:100C0000515CC8407047000040F2080041F2040106
:100C1000C2F20000C4F202010068096844F21062E6
:100C2000C1F3C221C0F60002515CC8407047000009
:100C30002DE9F04182B0002868D00446007841F2E6
:100C40000006C007C4F2020625D0706800F00C0050
:100C500004281BD0706800F00C00082802D17068CE
:100C6000C00313D46068002800F06881B0F5A02F9D
:100C700000F07C81B0F5803F00F07C81306820F48A
:100C800080303060306820F4802076E13068800366
:100C900001D56068D0B32078800718D5706810F04F
:100CA0000C0F07D0706800F00C0008286ED1706837
:100CB000C0036BD43068800702D52069012825D194
:100CC0003068616920F0F80040EAC10030602078A7
:100CD00000071FD42078400732D4E56995B17068C9
:100CE00000F00C00082840F08F80012D0ED07068B5
:100CF000216A00F480328A4208D1616A00F47010DF
:100D0000884203D1002002B0BDE8F081012002B08A
:100D1000BDE8F081A069002862D00020C4F2422022
:100D20000121C0F88014FFF7C1FD0546706A8007F5
:100D300000F18C80FFF7BAFD401B0228F6D92AE1AA
:100D4000F06910F0805808D1F06940F08050F061EF
:100D5000F06900F080500090009847F20007C4F25C
:100D600000073868C00529D4386840F480703860BE
:100D7000FFF79CFD054600BF3868C0051ED4FFF78D
:100D800095FD401B6428F7D905E100BF20690028C4
:100D900040F20000C4F2422000F082800121016094
:100DA000FFF784FD054600BF306880073FF588AF38
:100DB000FFF77CFD401B0228F6D9ECE0E068002834
:100DC00000F08080052800F09780012800F09880CE
:100DD000306A20F001003062306A20F0040092E0B6
:100DE0000020C4F242200021C0F88014FFF75EFD0D
:100DF000054600BF706A80077FF56CAFFFF756FDB0
:100E0000401B0228F6D9C6E00027C4F24227002082
:100E10003866FFF74BFD022D05460BD13068800187
:100E200040F1BE80FFF742FD401B02284FF0030057
:100E3000F4D968E7306880017FF564AFFFF736FDCD
:100E4000401B02284FF00300F4D95CE740F2080091
:100E5000C2F20000006844F6D351C1F26201A0FB67
:100E60000101480A019000BF00BF0198411E0028FF
:100E700001913FF42FAF00BF0198411E002801915E
:100E80003FF428AF00BF0198411E002801913FF4B4
:100E900021AF00BF0198411E00280191E4D119E75C
:100EA00000210160FFF702FD054600BF30688007A2
:100EB0007FF50DAFFFF7FAFC401B02284FF003004F
:100EC000F4D920E7306A20F001003062306A20F067
:100ED00004003062FFF7EAFC054641F2883700BFA4
:100EE000306A800720D5FFF7E1FC401BB8424FF085
:100EF0000300F5D907E700BF306A40F00400306214
:100F0000306A40F001003062FFF7D0FC054641F244
:100F1000883700BF306A800706D4FFF7C7FC401B44
:100F2000B842F7D937E000BFB8F1000F7FF4D5AE73
:100F3000F06920F08050F061CFE600BF306820F407
:100F400080303060306820F480203060FFF7AEFCE5
:100F5000054600BF306880037FF59DAEFFF7A6FC15
:100F6000401B64284FF00300F4D9CCE6306840F40D
:100F700080203060306840F480303060FFF796FCAD
:100F8000054600BF306880033FF585AEFFF78EFC55
:100F9000401B6428F6D9032002B0BDE8F08100BFF1
:100FA000206AB0F5803F05D17168A26821F4003154
:100FB000114371607168626A21F47411104308432F
:100FC000706001203866FFF771FC044630688001CC
:100FD0003FF598AEFFF76AFC001B02284FF00300B4
:100FE000F4D990E6411E0020B0EB116F1CBF012028
:100FF00070474EF21002CEF2000251604EF62351BD
:10100000CEF20001F0230B70072190601160704751
:1010100010B590F83C20012A4FF0020233D080F83E
:101020003D200268D2F804E0D2F808C00C682EF027
:101030007003234340F2FF74C4F20004A2425360E1
:101040000ADCB2F1804F13D040F20043C4F2000337
:101050009A420DD011E000BF42F60043C4F20103F2
:101060009A4205D040F60003C4F200039A4204D12C
:1010700049682CF08003194391600121002280F817
:101080003D1080F83C20104610BD0000002804BF31
:101090000120704710B5044690F83D0028B90020A3
:1010A00084F83C00204600F06FF8022084F83D00F0
:1010B000206840F2FF730268C4F2000342F6004C5D
:1010C0009842C4F2010C15DCB0F1804F1AD040F206
:1010D0000041C4F20001884214D0984218DCB0F1FB
:1010E000804F1DD040F20041C4F20001884217D069
:1010F0001AE000BF604505D040F60001C4F20001CF
:101100008842EAD1A16822F070020A439842E6DDE3
:10111000604505D040F60001C4F20001884203D1C9
:10112000216922F440720A43A36922F08001D4F8B5
:1011300004E0E268194360450160C262C0F828E03B
:1011400002D16169CCF83010012141610269D207F6
:1011500003D0026922F001020261002084F84610E7
:1011600084F83E1084F83F1084F8401084F8411051
:1011700084F8421084F8431084F8441084F8451031
:1011800084F83D1010BD000081B0006842F60041B7
:10119000C4F20101884201D001B0704741F2180049
:1011A000C4F20200016841F400610160006800F4CB
:1011B00000600090009801B07047000080B590F882
:1011C0003C20012A4FF0020200F0C28080F83D204E
:1011D000D0F800C04FF67772DCF8083023EA02023C
:1011E000CCF808200B684F2B28DC1F2B44DD202B6C
:1011F00045D0302B43D0402B40F0AC80D1F804E0F8
:10120000C968DCF82030DCF8202022F00102CCF89C
:101210002020DCF8182022F0F00242EA011123F02D
:101220000A0242EA0E02CCF81810CCF82020DCF8B2
:10123000081041F0470121F0300180E06F2B27DDDD
:10124000B3F5005F48D0B3F5805F7AD0702B40F0E3
:101250008180D1E901E3C968DCF8082043EA0E0384
:1012600022F47F4243EA01211143CCF80810DCF854
:10127000081041F0770162E00BB1102B6AD1DCF865
:10128000081021F07001194341F0070157E000BF39
:10129000502B35D0602B5DD1D1F804E0C968DCF863
:1012A0002030DCF8202022F01002CCF82020DCF8DE
:1012B000182022F4704242EA013123F0A00242EAEF
:1012C0000E12CCF81810CCF82020DCF8081041F0F1
:1012D000670121F0100132E0D1E901E3C968DCF8CF
:1012E000082043EA0E0322F47F4243EA012111431E
:1012F000CCF80810DCF8081041F480411FE000BF72
:10130000D1F804E0C968DCF82030DCF8202022F0B5
:101310000102CCF82020DCF8182022F0F00242EA8A
:10132000011123F00A0242EA0E02CCF81810CCF8A0
:101330002020DCF8081041F0570121F02001CCF802
:1013400008100022012180F83D10002180F83C1097
:10135000104680BD0122F5E72DE9F04390F83C30BE
:10136000012B04BF0220BDE8F0834FEAB202032A3A
:101370003CD8DFE802F003437FB900BF036842F6C0
:1013800000461D6A1A6AC4F2010622F001021A62BE
:101390001A465C6852F818CFB3428E68D1F800E064
:1013A00025F0020545EA06050CD1CE68D1E905789D
:1013B00024F4407425F00C0526F004063C43354324
:1013C00044EA08042CF0730747EA0E075C609F614B
:1013D0004F6809695F631D629F6947F008079F6155
:1013E0009F6927F004079F61AEE000BF0121002242
:1013F00080F83C200846BDE8F08300BF036842F651
:1014000000461D6A1A6AC4F2010622F010021A622E
:101410001A46D3F804C052F8184FB3428E68D1F878
:1014200000E025F0200545EA06150FD1CE68D1E988
:1014300005986FF0400707EA06162CF4406725F080
:10144000C00547EA8907354347EA880C24F4E64497
:1014500044EA0E27C3F804C09F614F6809699F637F
:101460001D629F6947F400679F619F6927F4806749
:101470009F6168E0036842F600461D6A1A6AC4F27A
:10148000010622F480721A621A46D3F804C052F898
:101490001CEFB3428E680C6825F4007545EA0625FA
:1014A0000FD1CE68D1E90598360240F2FF47BE431E
:1014B0002CF4405725F4406547EA0917354347EABD
:1014C000081C2EF073072743C3F804C0DF614F6880
:1014D0000969DF631D62DF6947F00807DF61DF69C3
:1014E00027F00407DF612FE0036842F60047D3F8D6
:1014F00020C01A6AC4F2010722F480521A621A4606
:101500005C6852F81C5FD1F800E08E68BB4204D1E1
:101510004F6924F4804444EA87142CF4005747EAC6
:10152000063725F4E64646EA0E265C60DE614E6824
:1015300009691E641F62DF6947F40067DF61DF69C4
:1015400027F48067DF6109021368194311600021E5
:10155000002280F83C200846BDE8F083002804BF44
:101560000120704710B5044690F83D0028B90020CE
:1015700084F83C00204600F06FF8022084F83D001B
:10158000206840F2FF730268C4F2000342F6004C88
:101590009842C4F2010C15DCB0F1804F1AD040F231
:1015A0000041C4F20001884214D0984218DCB0F126
:1015B000804F1DD040F20041C4F20001884217D094
:1015C0001AE000BF604505D040F60001C4F20001FA
:1015D0008842EAD1A16822F070020A439842E6DD0F
:1015E000604505D040F60001C4F20001884203D1F5
:1015F000216922F440720A43A36922F08001D4F8E1
:1016000004E0E268194360450160C262C0F828E066
:1016100002D16169CCF83010012141610269D20721
:1016200003D0026922F001020261002084F8461012
:1016300084F83E1084F83F1084F8401084F841107C
:1016400084F8421084F8431084F8441084F845105C
:1016500084F83D1010BD000081B00068B0F1804FEB
:1016600002D001B0704700BF41F21C00C4F202007A
:10167000016841F001010160006800F00100009084
:10168000009801B07047000041B1082910D004292A
:1016900014BF00F1410200F13F020BE090F83E2040
:1016A000012A1CBF01207047022280F83E2013E06F
:1016B00000F140021278012A1CBF0120704702226B
:1016C000082907D0042914BF80F8412080F83F2062
:1016D00002E000BF80F84020006801F01F010122F5
:1016E000036A8A4023EA02010162036A42F6444126
:1016F000C4F201011A43A1F14403984202620FD0DF
:1017000040F2FF71C4F20001884213DCB0F1804F57
:101710001CD040F20041C4F20001884216D01CE007
:101720000A6842F400420A6040F2FF71C4F200010C
:101730008842EBDD42F60041C4F20101884205D047
:1017400040F60001C4F20001884206D1816801F030
:101750000701062904BF00207047016841F001011C
:1017600001600020704700007047000070470000D3
:10177000B0B582B0056804462968EA68686901F076
:101780002F03202B02F0200306D12BB1204602B0FC
:10179000BDE8B04000F038BF5FEA017C1EBF00F03A
:1017A000010E02F4907010EB0E002FD1236B02EAB1
:1017B0000100C10618D5012B16D100200190286820
:1017C00001906868019001986869400628D4A08D4E
:1017D000E18DE28D002A1CBF411A5FEA014040F012
:1017E000D78102B0B0BD00BF010600F1D380400632
:1017F000F7D5E868202120F04000E860204684F812
:10180000411002B0BDE8B04000F026BCC80718BFC8
:1018100012F4807040F0D280480700F1D580DAE001
:10182000E06B01684A6893B2002BDAD0A18D8B423D
:10183000D7D2E2858069202800F0A18055E8030F07
:10184000216820F4807041E80302FAB1206850E872
:10185000030F216820F4807041E80302B2B12068D0
:1018600050E8030F216820F4807041E803026AB158
:10187000206850E8030F216820F4807041E80302DB
:1018800022B1206850E8030FDAE700BF206850E873
:10189000050F216820F0010041E80502BAB3206875
:1018A00050E8050F216820F0010041E8050272B3FD
:1018B000206850E8050F216820F0010041E805028A
:1018C0002AB3206850E8050F216820F0010041E8A4
:1018D0000502002ADAD11AE0206850E8050F2168D5
:1018E00020F0400041E80502DAB1206850E8050F19
:1018F000216820F0400041E8050292B1206850E8DC
:10190000050F216820F0400041E805024AB1206837
:1019100050E8050F216820F0400041E80502002A48
:10192000DAD1202084F8420000202063206850E8AB
:10193000030F216820F0100041E80302DAB12068AB
:1019400050E8030F216820F0100041E8030292B133
:10195000206850E8030F216820F0100041E80302DE
:101960004AB1206850E8030F216820F0100041E8D8
:101970000302002ADAD1E06BFEF788FCA18D022079
:101980006063E08D081A81B2204602B0BDE8B04025
:10199000FFF7EABE94F8410021287FF422AFA06847
:1019A000B0F5805F03D12069002800F08981206AAA
:1019B000411C21620078686089E100BF606C40F0E2
:1019C00001006064480706D5BEF1000F03D0606CCB
:1019D00040F002006064880706D5BEF1000F03D016
:1019E000606C40F004006064BCF1000F06D55EEA54
:1019F000030003D0606C40F008006064606C002855
:101A00003FF4EFAE02EA0100800603D5204600F065
:101A1000FBFD25686869616C00F0400001F0080179
:101A2000401800F0AD8055E8030F00BF216820F496
:101A3000907041E80302D2B3206850E8030F216898
:101A400020F4907041E803028AB3206850E8030F45
:101A5000216820F4907041E8030242B3206850E806
:101A6000030F216820F4907041E80302FAB1206866
:101A700050E8030FDAE700BF206850E8050F21683F
:101A800020F0010041E80502DAB1206850E8050FB6
:101A9000216820F0010041E8050292B1206850E879
:101AA000050F216820F0010041E805024AB12068D5
:101AB00050E8050F216820F0010041E80502002AE6
:101AC000DAD1206B012824D1206850E8030F216867
:101AD00020F0100041E80302DAB1206850E8030F5B
:101AE000216820F0100041E8030292B1206850E81C
:101AF000030F216820F0100041E803024AB120687A
:101B000050E8030F216820F0100041E80302002A8A
:101B1000DAD1202084F84200002020632068416947
:101B2000490640F1C78050E8050F216820F04000C9
:101B300041E80502002A00F0AB80206850E8050F5C
:101B4000216820F0400041E80502002A00F0A08052
:101B5000206850E8050F216820F0400041E80502A8
:101B6000002A00F09580206850E8050F216820F0D9
:101B7000400041E80502002A00F08A802068D2E790
:101B80002046FFF7F3FD0020606402B0B0BD00BF47
:101B900055E8030F226820F4907042E80303D3B3A2
:101BA000206850E8030F226820F4907042E8030395
:101BB0008BB3206850E8030F226820F4907042E84D
:101BC000030343B3206850E8030F226820F49070A9
:101BD00042E80303FBB1206850E8030FDAE700BFD7
:101BE000206850E8050F226820F0010042E8050354
:101BF000DBB1206850E8050F226820F0010042E8C0
:101C0000050393B1206850E8050F226820F0010019
:101C100042E805034BB1206850E8050F226820F028
:101C2000010042E80503002BDAD1202084F84200AD
:101C300000202063206850E8030F226820F0100085
:101C400042E80303DBB1206850E8030F226820F06C
:101C5000100042E8030393B1206850E8030F2268A4
:101C600020F0100042E803034BB1206850E8030F56
:101C7000226820F0100042E80303002BDAD1022290
:101C800089B22046626302B0BDE8B040FFF76CBD88
:101C9000E06B78B142F20931C0F600014163FEF712
:101CA00019FB00283FF49DADE06B416B02B0BDE82D
:101CB000B0400847204602B0BDE8B040FFF756BD2F
:101CC000206A30F8021B6FF35F2169602062E08CAC
:101CD00001380104E0847FF484ADE86820F08000DE
:101CE000E860E86840F04000E86002B0B0BD000085
:101CF000002804BF0120704710B5044690F8410049
:101D000028B9002084F84000204600F061F8242023
:101D100084F841002068D4E90212C36823F4005318
:101D2000C360036923F440531A430261D4E90423D6
:101D30001143C268194341F20C639A431143C160D5
:101D40004169A26921F44071114343F60002C4F2D3
:101D500001029042416103D0FEF742FF02E000BF62
:101D6000FEF752FF6268192148439100B0FBF1F081
:101D700048F21F51C5F2EB11A0FB01235A096FF085
:101D8000630302FB0300322303EB0010A0FB0101FD
:101D9000F02303EA5113206803EB0212C1F343114D
:101DA00011448160016921F490410161416921F090
:101DB0002A014161C16841F40051C1600020202125
:101DC000606484F8411084F84210606310BD000024
:101DD0002DE9F04186B040F600050446C4F2010545
:101DE0000068A5F5444100278842049702D006B058
:101DF000BDE8F08141F21800C4F20200416802AE71
:101E000041F400314160416840F26C0801F4003156
:101E1000019101990168C4F2020841F004010160D6
:101E20000068314600F004000190019804200290FF
:101E300002200390032005902846FEF727FC082087
:101E4000CDE90207284631460497FEF71FFC40F211
:101E5000D405C2F2000580262846C5E90087C5E9F9
:101E60000276C5E90477C5E90677FEF769FB002825
:101E700018BFFEF705FAE5636C6240F2181508F129
:101E80001400C2F200051021002285E84700284610
:101E9000C5E90422C5E90622FEF752FB002818BF57
:101EA000FEF7EEF9262000210022A5636C62FEF702
:101EB0007BFD2620FEF768FD06B0BDE8F08100003E
:101EC00070B582B0044690F8420020280AD113462B
:101ED0000A4600294FF0010018BF002B06D102B0BE
:101EE00070BD00BF022002B070BD00BF00252220DF
:101EF0002563A262A385656484F842002168E06BD3
:101F000042F2914C42F2F15E42F21536C0F6000CFC
:101F1000C0F6000EC0F600060431C0E90ACEC0E9E2
:101F20000C65FEF751FB019520680168019141683D
:101F300001910199216929B350E8030F216840F408
:101F4000807041E80302EAB1206850E8030F21687D
:101F500040F4807041E80302A2B1206850E8030F0A
:101F6000216840F4807041E803025AB1206850E8CB
:101F7000030F216840F4807041E8030212B1206829
:101F8000DAE700BF206850E8050F216840F0010043
:101F900041E80502BAB3206850E8050F216840F017
:101FA000010041E8050272B3206850E8050F21687E
:101FB00040F0010041E805022AB3206850E8050F0F
:101FC000216840F0010041E80502002ADAD11AE058
:101FD000206850E8050F216840F0400041E8050204
:101FE000DAB1206850E8050F216840F0400041E870
:101FF000050292B1206850E8050F216840F04000CA
:1020000041E805024AB1206850E8050F216840F018
:10201000400041E80502002ADAD1002002B070BD7C
:10202000006844F20041C4F20001884218BF7047C2
:1020300040F2700C40F2EC1040F29801C2F2000C39
:102040000123C2F20000C2F2000119228CF8003014
:10205000FFF736BF7047000070470000FEE7000042
:1020600080B582B041F21400C4F20200016800227F
:1020700041F0010101600068002100F001000190C1
:1020800001981020FEF790FC1020FEF77DFC112037
:1020900000210022FEF788FC112002B0BDE880403C
:1020A000FEF772BC70B584B041F21800C4F20200B1
:1020B000016840F6004441F0100101600168C4F27B
:1020C000010401F01001009100990168002241F023
:1020D0002001016001684FF4704501F0200100917A
:1020E00000990168002641F004010160016801F0D7
:1020F000040100910099016841F008010160006845
:102100004FF4704100F00800009000982046FEF760
:10211000C7FB0120CDE90106022003906946204655
:102120000095FEF7B3FA04B070BD000080B586B02C
:1021300040F25C1042F600420021C2F20000C4F2FC
:10214000010247234FF0630C4FF0800E0591CDE95B
:102150000311CDE90011C0E90023C0E9021CC0E968
:102160000411C0F818E0FEF791FF002818BFFEF731
:1021700087F84FF48050029040F25C10C2F20000E9
:1021800002A9FFF71BF8002818BFFEF779F8002016
:10219000CDE9000040F25C10C2F200006946FEF793
:1021A00037FF002818BFFEF76BF806B080BD0000AF
:1021B00010B590B040F2A4100021C2F200004FF020
:1021C0008042472363240991CDE90711CDE9051128
:1021D000CDE90311CDE90111C0E90023C0E90214E2
:1021E00001618161FFF7BAF9002818BFFEF748F8CE
:1021F00040F2A410C2F2000008A9FEF709FF00286F
:1022000018BFFEF73DF8602001900020CDE90200E4
:10221000059040F2A410C2F2000001A90822FFF7C5
:102220009BF8002818BFFEF72BF840F2A414C2F266
:10223000000401A920460C22FFF78EF8002818BFE1
:10224000FEF71EF820680021B0F1804F0E9101D0FA
:1022500010B010BD41F21800C4F20200016841F054
:102260000801016000680CA900F008000B900B98B1
:102270004FF440600C9002200D900F9040F600400B
:10228000C4F20100FEF702FA0420C4F20100016862
:102290004FF6FF42CFF6FF02114041F0E06141F4FA
:1022A0000071016010B010BD80B540F2EC1044F236
:1022B000004C48F2A062C2F20000C4F2000CC0F26E
:1022C00001024FF4805300214FF00C0EC0E900C210
:1022D000C0E90231C0E9041EC0E90611FFF708FD9C
:1022E000002808BF80BDBDE88040FDF7C9BF0000E1
:1022F000FEE70000FEE700007047000070470000A6
:10230000FEF7DABA70470000406A0021C185C18437
:10231000FFF72CBA406A01684A6990F84130212BD6
:102320002ED112F080022BD00022C28451E8031F6C
:10233000026821F0C00142E80313EBB1016851E8E3
:10234000031F026821F0C00142E80313A3B1016832
:1023500051E8031F026821F0C00142E803135BB19A
:10236000016851E8031F026821F0C00142E803132D
:1023700013B10168DAE700BF202180F8411001683D
:102380004A6990F84230222B7CD112F0400279D079
:102390000022C28551E8031F026821F4907142E8CF
:1023A0000313C3B3016851E8031F026821F490715D
:1023B00042E803137BB3016851E8031F026821F46C
:1023C000907142E8031333B3016851E8031F0268B8
:1023D00021F4907142E80313EBB10168DAE700BF22
:1023E000016851E8051F026821F0010142E8051368
:1023F000DBB1016851E8051F026821F0010142E8E4
:10240000051393B1016851E8051F026821F001012D
:1024100042E805134BB1016851E8051F026821F03D
:10242000010142E80513002BDAD1016B012924D107
:10243000016851E8031F026821F0100142E803130C
:10244000DBB1016851E8031F026821F0100142E886
:10245000031393B1016851E8031F026821F01001D2
:1024600042E803134BB1016851E8031F026821F0F1
:10247000100142E80313002BDAD1202180F842102A
:1024800000210163416C41F010014164FFF76EB916
:102490000168406A0968890600F19F800021C185B2
:1024A000016851E8031F026821F4807142E80313B8
:1024B000E3B1016851E8031F026821F4807142E82A
:1024C00003139BB1016851E8031F026821F4807176
:1024D00042E8031353B1016851E8031F026821F475
:1024E000807142E80313002BDAD100BF016851E884
:1024F000051F026821F0010142E80513BBB3016822
:1025000051E8051F026821F0010142E8051373B389
:10251000016851E8051F026821F0010142E8051336
:102520002BB3016851E8051F026821F0010142E860
:102530000513002BDAD11AE0016851E8051F026883
:1025400021F0400142E80513DBB1016851E8051FA5
:10255000026821F0400142E8051393B1016851E897
:10256000051F026821F0400142E805134BB10168E4
:1025700051E8051F026821F0400142E80513002BD5
:10258000DAD1202180F84210016B012925D100BF4A
:10259000016851E8031F026821F0100142E80313AB
:1025A000DBB1016851E8031F026821F0100142E825
:1025B000031393B1016851E8031F026821F0100171
:1025C00042E803134BB1016851E8031F026821F090
:1025D000100142E80313002BDAD100214163016BA3
:1025E000012918BFFFF71CBD818DFFF7BDB80000A2
:1025F000406A01214163016B012918BFFFF72ABD21
:10260000818D4908FFF7B0B881B090F842102229B7
:1026100020D18368B3F5805F08D10169002957D0C4
:1026200000F128010A6803685B680AE0014651F876
:10263000282F13B90369002BF5D003685B6803F0FA
:102640007F0313700A6801320A60C18D01390A04E0
:10265000C18501D001B070470168CA6822F020022C
:10266000CA60CA6822F48072CA604A6922F0010214
:102670004A61202280F8422000224263036B012B32
:1026800030D1026351E8031F026821F0100142E8D3
:1026900003135BB3016851E8031F026821F01001C6
:1026A00042E8031313B3016851E8031F026821F0E5
:1026B000100142E80313CBB1016851E8031F02681F
:1026C00021F0100142E8031383B10168DAE700BF8B
:1026D0000168826A49686FF35F2122F8021B8262F7
:1026E000B3E700BF01B0FFF79BBC00BF01680A68F9
:1026F000D20606D5002200920A680092496800912D
:102700000099818D01B0FFF72FB8000040F2EC1066
:10271000C2F20000FFF72CB8FEE70000F0B581B070
:1027200040F27007C2F20007B7F94800C82100FB69
:1027300001F24AF6C003D21A48F29D23C5F297333C
:1027400082FB0323B7F946204EF2C066CFF6FE7631
:1027500002FB016148F21F56C5F2EB167880581251
:1027600081FB061600EBD370A0F16404701200EB3D
:10277000D6706438BA80C7E9044001F056FA0546BD
:1027800020460E4601F051FA02460B4628463146D5
:1027900000F04CFE00F068FF0446F868BC6001F0F1
:1027A00044FA054620460E4601F062FC7A2242F2C7
:1027B000FA13CFF68B42CBF6E97300F087FF00F0F7
:1027C00003FF2A46334601F05BFA00F04DFF00217B
:1027D0000446B86101F085FC40F60045C4F20105ED
:1027E0004FF40051002828464FF0010218BF4FF463
:1027F0008051FEF755F82046002101F072FC4FF49D
:102800008051002828464FF0000218BF4FF40051B5
:10281000FEF746F82046002101F063FC4FF400412A
:10282000002828464FF0010218BF4FF48041FEF700
:1028300037F82046002101F054FC4FF48041002875
:1028400028464FF0000218BF4FF40041FEF728F869
:10285000B86920F0004001F0A1FC40F2A411C2F2DE
:1028600000010968C863086401B0F0BD90B0FEF7CC
:1028700031F800240120CDE90B44CDE9094406904C
:102880000A904FF4E0104FF4803102250F9006A813
:102890000594CDE90344CDE90144CDE90714CDE920
:1028A0000D51FEF7C5F928B1EFF3108072B600BFE5
:1028B000FEE700BF0F20CDE901054FF48060CDE9B0
:1028C000040401A802210394FEF7AAF820B1EFF353
:1028D000108072B6FEE700BF40F60048C4F201085F
:1028E000FFF7E0FBFFF7BCFBFFF7DEFCFFF760FC48
:1028F000FFF71CFC40F27007C2F2000707F1280541
:1029000040F2EC10C2F2000029461922FFF7D8FA73
:1029100040F2A416C2F2000630460821FEF7B4FECB
:1029200030460C21FEF7B0FE4FF0500A4FF00A0976
:10293000002407F1420602E04B20FDF793FE3878B1
:1029400020B12846314600F04DF83C70B7F84A10E7
:10295000B7F84C00C82908BFC82827D0C82908BF25
:10296000B0F57A7F34D0C82908BFB0F5E16F21D126
:1029700040464FF480510022FDF792FF40464FF44D
:1029800000510022FDF78CFF40464FF480410022A9
:10299000FDF786FF40464FF400410022FDF780FF1F
:1029A000B7F84A00B0F57A7F09D0C5E7C7F80CA0A0
:1029B000FFF7B4FEB7F84A00B0F57A7FBCD1B7F89C
:1029C0004C00B0F57A7FB7D100F088F8B4E700BFCB
:1029D000C7F80C90FFF7A2FEB7F84A00B0F57A7F6F
:1029E000EDD0A9E702780F2A18BF704742788378A4
:1029F00063F30A220A808278C378D20863F34A120A
:102A00004A80037990F803C042799B0043EA9C1303
:102A100002F0010243EA82228A80427983795208D5
:102A200063F3CA12CA808279C379120963F30A1266
:102A30000A81037A90F807C0427A5B0043EADC130C
:102A400002F0030243EA42224A81427A837A9208E0
:102A500063F38A128A81C27A837AD20042EA5312DD
:102A6000CA81027B437B63F30A220A82427B837B17
:102A7000D20863F34A124A82C37B90F80EC0027CEC
:102A80009B0043EA9C1302F0010243EA82228A82FD
:102A9000027C437C520863F3CA12CA82427C837C64
:102AA000120963F30A120A83C37C90F812C0027DF4
:102AB0005B0043EADC1302F0030243EA42224A834A
:102AC000027D437D920863F38A128A83827D407D72
:102AD000D20042EA5010C883704700002DE9F0414F
:102AE00040F27008C2F20008B8F842004AF600410D
:102AF00000EB8000CFF6FE7101EB40104EF21D217D
:102B0000C5F22A3180FB0101081200EBD170503868
:102B100001F08BF8D8F81C20C8E9080102F10E0377
:102B20001C2B03D80020C8F81C000BE0002A09DD8C
:102B30004FF400444FF480454FF480564FF4005159
:102B400008E000BF4FF480444FF400454FF40056B6
:102B50004FF4805140F60047C4F201073846012285
:102B6000FDF79EFE384631460022FDF799FE3846B5
:102B700029460122FDF794FE384621460022FDF742
:102B80008FFED8E9080121F0004101F021F840F260
:102B9000A411C2F200010968C8630864BDE8F081AD
:102BA000490050EAC12018BF04204A0D18BF40F068
:102BB000010040F2FF72B2EB515F08BF40F002002B
:102BC000012808BF052070472DE9F74F144694B03F
:102BD0000021C4E902111599079121F00045C94966
:102BE0008D4206DC1599C4E9000117B00020BDE84C
:102BF000F08FC549DFF814A3A9423CDD0799C44E04
:102C00000029C44FC44A1599534619DD01F042F911
:102C1000554506D0C14AC24B01F03CF9C4E9000158
:102C20000AE04FF0D352BE4B01F034F932463B4636
:102C300001F030F9C4E9000117B00120BDE8F08FC0
:102C400000F044FD554506D0B44AB54B00F03EFDBA
:102C5000C4E900010AE04FF0D352B14B00F036FD59
:102C600032463B4600F032FDC4E9000117B04FF098
:102C7000FF30BDE8F08FAB49A942159978DB21F010
:102C8000004183468846A84AA84B00F0F9FF00227D
:102C9000A74B00F01BFD00F06BFF099000F0C5FF93
:102CA00006460F469C4A534600F0EAFF43465A4602
:102CB00001F0E4F880468A46984A994B30463946F6
:102CC00000F0DEFF2A0D01250B924246534601F02B
:102CD000D5F8032DC4E9000139D00B98C1F30A518E
:102CE000401A05EB45111139814230DA9148C3464B
:102CF000784400EB0510CDF80CA00C90D0E900232F
:102D00003046394600F0BCFF02460B46049106905F
:102D10005846039901F0BEF880468A4602460B46A3
:102D20005846039901F0B6F8049B069A01F0B2F8F0
:102D300083460C9803913946D0E90223304600F0CF
:102D40009FFF5A46039B01F0A5F86D1CBDE707984D
:102D50000028A2BF099817B0BDE8F08F616881F024
:102D600000416160099817B04042BDE8F08FFFE76D
:102D700084461598C1F31301C0F30A50A0F2F53050
:102D80004FEA601800F01F06C6F1200013900020E3
:102D90000690079041F4801E05206D4676B1664A84
:102DA00008EB00017A4452F8213002EB8101B34074
:102DB0004A68139922FA01F1194305E05F4908EBCB
:102DC0000002794451F82210A1FB0E27A1FB0C133D
:102DD0001A449A4234BF0123002303EB070A05EB90
:102DE0008003D3E901B70F448F4234BF0121002192
:102DF00093448B4411B1934502D903E0934501D22A
:102E0000012100E00021C3E901B7514445F8201039
:102E1000011EA0F10100C1DC0298059F00F10050E5
:102E2000800F12900298DDE90356800000F0FDFE4D
:102E3000834628460D9100F00FFF6FF01D0201F050
:102E4000B2FACDE90E01304600F006FF6FF03D0208
:102E500001F0A9FA80468A46384600F0FDFE6FF080
:102E60005D0201F0A0FA074642465346119100F078
:102E70002DFCDDE90E2300F029FC5A460D9B00F0E5
:102E800025FC00250E465A4628460D9B01F002F807
:102E9000DDE90E2300F0FEFF4246534600F0FAFF44
:102EA0003A46119B00F0EAFFDFF898A0244A534607
:102EB00000F0E6FE07468846234A244B3146284662
:102EC00000F0DEFE3A46434600F000FC0746884626
:102ED0004FF0A84253463146284600F0D1FE3A460C
:102EE000434600F0F3FB159A12F0004F04D0129AFB
:102EF00081F0004152421292C4E90001129817B0C9
:102F0000BDE8F08FFB21E93F7CD90240FB21F93F6E
:102F10007370032E8A19A33B000040543163621A78
:102F200061B4D03DFB21394183C8C96D305FE43FB6
:102F30000000E03F14180000901700007217000016
:102F4000182D4454FB21F93D3326A611460B113CA4
:102F50002DE9FF4D21F0004807460C46B8F1795F96
:102F600008DA00F005FE002801BF0020324904B055
:102F7000BDE8F08D3A4623461046194600F080FE23
:102F8000054602462D480E460B460621784400F0C1
:102F90005DF82A46334600F073FEDDE902238246DF
:102FA0008B463846214600F06BFE04460F465246DB
:102FB0005B462846314600F063FE22463B4600F061
:102FC00069FF07468A464FF0FF322846314601F036
:102FD000EAF91B4A90450ADA3A46534600F05AFF8E
:102FE00004B00022BDE8F04D134B00F047BF154A76
:102FF0004245A8BFA8F500154FF00004B8BF124D18
:1030000022462B4600F046FF0646884622462B46BF
:103010000020094900F03EFF04460D463A4653465B
:103020003046414600F036FF04B022462B46BDE84C
:10303000F04D00F023BF00000000F03F40150000FD
:103040003333D33F0000E93F0000D23F2DE9F04188
:103050004F1E00EBC7010446D1E9000115461E468C
:1030600037F006020DD02A46334600F009FE7F1ED7
:1030700004EBC703D3E9002300F028FB37F0060276
:10308000F1D1022F25D0042F13D0062F18BFBDE891
:10309000F0812A46334600F0F3FDD4E90A2300F01C
:1030A00015FB2A46334600F0EBFDD4E9082300F077
:1030B0000DFB2A46334600F0E3FDD4E9062300F079
:1030C00005FB2A46334600F0DBFDD4E9042300F07B
:1030D000FDFA2A46334600F0D3FDD4E9022300F07E
:1030E000F5FA2A46334600F0CBFDD4E90023BDE8CB
:1030F000F04100F0EBBA00002DE9FF4D054621F04C
:10310000004084B00C46B0F1795F0BDA2846FFF737
:1031100047FD042808BF00F071F8284608B0214692
:10312000BDE8F08D2A460B46104600F0A9FD064684
:103130000F462A46234600F0A3FD804626488A46CD
:1031400032463B4605217844FFF780FF83461098BE
:10315000029160B3214A224B4046514600F090FD57
:10316000CDE900015A4640465146029B00F088FDD9
:1031700082468846DDE906014FF0FF3201F013F97F
:103180005246434600F086FE32463B4600F078FD4C
:10319000DDE9062300F07EFEDDE9002300F07AFE83
:1031A00008B02A462346BDE8F04D00F067BE0B4646
:1031B0005A463046394600F063FD084A084B00F095
:1031C00085FA4246534600F05BFD08B02A46234686
:1031D000BDE8F04D00F07ABA8E14000049555555FF
:1031E0005555C5BF012201F0DEB800F06FBA0022CC
:1031F00013461046114600F025BB0000024A00208D
:10320000110701F0D0B8000001FDFFFF2DE9F84FD4
:1032100004460D4621F0004000917349814211DCC3
:103220007249884201DC06D12CB120462946BDE80E
:10323000F84FFFF7D7BF6E48002DCCBF6D496E49E0
:10324000BDE8F88F6D49814211DD6D498142D8BFDB
:103250004FF0FF366DDD20462946FFF7A1FC04281C
:1032600008BFFFF7CBFF20462946BDE8F88F654928
:10327000654F25F00045814233DD6449814219DD07
:10328000002632464FF080432046294600F01EFAC1
:1032900080468A4601222046294601F084F8002211
:1032A0003B4600F0F7FD4246534600F0CBFA044699
:1032B0000D463EE001260022BA463B4620462946FE
:1032C00000F004FA80460F46002253462046294665
:1032D00000F0E0FD42463B4600F0B4FA04460D46DD
:1032E00027E04B4981421BDDDFF828A1022600229E
:1032F00053462046294600F0C3FC00223B4600F01E
:10330000E5F980460F46002253462046294600F044
:10331000C1FD42463B4600F095FA04460D4608E0E2
:10332000032622462B4600203B4900F08BFA044638
:103330000D4622462B461046194600F0A1FC8B464E
:10334000824602460B4600F09BFC07460246334885
:1033500088460B4606217844FFF778FE52465B46C6
:1033600000F08EFC82462E488B463A4643460521A5
:103370007844FFF76BFE3A46434600F081FC024674
:103380000B46002E504659460CDA00F09FF92246B3
:103390002B4600F075FC01B022462B46BDE8F04FED
:1033A00000F06CBD00F092F922462B4600F068FC5C
:1033B0001C4A7A4402EBC603D3E9002300F06AFDFD
:1033C00022462B4600F066FD174A7A4402EBC603FC
:1033D000D3E9002300F052FD009A002AB8BF81F023
:1033E0000041BDE8F88F0000000010440000F07FAD
:1033F000182D4454FB21F93FFB21F9BF0000DC3FAD
:103400000000203E0000F33F0000F03F0000E63FD8
:10341000008003400000F83F0000F0BF46110000AC
:1034200004110000A21000006A1000002DE9F04D08
:103430009446CCF1000423F000464CEA0404594FB2
:1034400046EAD4749A46884621F00042BC4206D827
:10345000454240EA050442EAD474BC4204D9BDE8BE
:10346000F04D6246FFF7C1BEAAF14055A5F17F6558
:1034700055EA0C040BD0022404EAAA744A4DDFF882
:103480002CE144EAD87452EA000B04D00CE0BDE809
:10349000F04DFFF7BBBE002C14BF012CBDE8F08D32
:1034A000022C30D0032C32D056EA0C0B0AD0BE428C
:1034B00020D1BA4209D126F0804622F0804233461C
:1034C000114617E000291ADB25E0DFF8E4B0FB44E1
:1034D000002C04BFDBE90001BDE8F08D012C02BF28
:1034E000DBE9000181F00041BDE8F08D022C0AD03B
:1034F000032C0CD0BA4212D1B8F1000F0BDA2A48D3
:103500002C49BDE8F08D28462B49BDE8F08D2846B2
:103510007146BDE8F08D24482849BDE8F08D921B26
:1035200012153C2AC4BF204F244E10DCBAF1000F04
:10353000BEBF12F13C0F00273E4608DB624600F09A
:1035400081F921F00041FFF761FE07460E4694B174
:10355000012C08BF86F000460DD0194A194B022CE9
:103560003846314615D000F095FC2A46BDE8F04DAE
:10357000114B00F08FBC002213463846314600F054
:10358000BBFA04BF0220FCF727FE38463146BDE8EF
:10359000F08D00F07FFC2A46BDE8F04D064B00F0B0
:1035A0006DBC00000000F07F182D4454FB2109C0C1
:1035B0002E100000FB21F9BFFB210940FB21F93F40
:1035C000075C143326A6A13C00B5254B21F0004230
:1035D00087B09A4203DC0022134600922BE0214B75
:1035E0009A4208D140B94FF00100FCF7F5FDFFF712
:1035F000FEFD07B000BD03DBFFF7F4FD07B000BD23
:1036000002AAFFF7E1FA10F003014FF001000DD01C
:10361000012914D002291AD00DF1080C9CE80F00E2
:10362000FFF796FC07B081F0004100BD0DF1080CDA
:1036300000909CE80F00FFF75FFD07B000BD0DF1A3
:10364000080C9CE80F00FFF783FC07B000BD0DF1EC
:10365000080C00909CE80F00FFF74EFDE2E7000029
:10366000FB21E93F0000F07F21F0004201F0004320
:10367000A2F16052B2F5801F28BFD2F17F6C0BD946
:103680005FEA001C43EAC20242EB507018BF704769
:1036900028BF20F001007047B2F5801FBCBF18465C
:1036A00070474FEA410C1CF5001F02D2084600F09B
:1036B00043BE70B500F08EFB00000089FFF7F6BF37
:1036C0004FF00040A0F580007047000010B591EA6F
:1036D000030F48BF83F0004300F1E483841A71EBC9
:1036E000030C05D2121943EB0C03001B61EB0C0118
:1036F0004FEA1154A4EB135CDFF81CE11EEA430F00
:1037000018BF9EEA445F00F0748021EA045123EA66
:103710000E0343F48013DCF1200E32D322FA0CFEA8
:1037200010EB0E0023FA0CFE41EB0E01CCF1200E43
:1037300003FA0EFE10EB0E00CCF1200E51F1000149
:10374000B1F5801F32D201EB045112FA0EF2BDE83E
:10375000104058BF7047401C38BF5FEA420218BF94
:103760007047002814BF20F0010041F100014FEA2A
:10377000410313F5001F38BF7047A1F1C04100F0AD
:1037800077BB012A43EB0302ACF1200CDCF11F0EE6
:1037900032BF4FF0000E23FA0CF310EB030041EBA5
:1037A0000451B4EB115FD0D0A1EB045101F58011AD
:1037B000490801EB04515FEA30000ED350F10000DC
:1037C00038BF12FA0EFE08D1BDE81040C9E7401C10
:1037D00038BF5FEA4202CAD1C3E7BDE810404FEAF2
:1037E000410313F5001F38BF7047A1F1C04100F03D
:1037F0003FBB9EEA445F08D011EA5E0FBDE810406F
:1038000004BF01F0004100207047BDE8104070B5D2
:1038100000F0E0FA64FBBE3E0000E0FF02494FF01A
:10382000000000F08EBD00BF0000F87F491058BFB7
:10383000C1F140415B1058BFC3F140438B42EFF3ED
:10384000008070472DE9C04130B4DFF8A4C23CEAE3
:10385000111418BF3CEA131400F0ED801CEA111497
:1038600081EA030544EAD57418BF1CEA131500F079
:10387000C880A4EB050404F17F7404F500344FF014
:10388000004545EAC12145EAC32341EA505143EAD4
:1038900052534FEAC0204FEAC222994208BF9042D9
:1038A00000F09D804FEA13650FF24416765D4FEAF3
:1038B000134506FB05F7C7F1807706FB07F74FEACC
:1038C000D737A7FB03687642A7FB06CEC8F580383A
:1038D00038BFA8F1010807FB08E6A6FB028C4FF0F1
:1038E000000EE6FB03CEDCF1000CCEF1004E38BF3B
:1038F000AEF1010EA6FB0C584FF00007E6FB0E8759
:10390000A1FB08C6A0FB07CE16EB0E064FF0000584
:1039100045F10005E1FB076515F1E04E7EBFA4F51A
:1039200080345FEA46066D4116F1800745F10005D7
:103930004FEA172747EA05674FEA15254FEA06665B
:10394000A6F1DE46B6F1805F20D9384605EBC4719A
:1039500024F0010C01EB0C11BCF1FE6F02D8F0BC9D
:10396000BDE8008124425CBF01F5801E9EEAC47F51
:1039700002D4F0BCBDE80081244200F13980A1F1FD
:10398000C041F0BCBDE8004100F072BA4FEAD0205F
:1039900040EA41504FEAD1214FEAD22242EA435253
:1039A0004FEAD323A7FB028607FB036605FB0266EB
:1039B0001EEA0E0F58BFA6EB0056B6EB00564FEAB4
:1039C000520E4EEAC37E18EB0E0E56EB530EBCD5CC
:1039D00018EB02085E417F1C55F10005B5E74FF476
:1039E00080154FF000074FF000064FF00008ACE7DD
:1039F00001F1C04101F000414FF00000F0BCBDE812
:103A000000810CEA131511EA0C1F00D00CE013EA38
:103A10000C1F00F026804FF0000081EA030101F046
:103A20000041F0BCBDE80081F0BCBDE8004181EA86
:103A3000030100F01DBAF0BCBDE8004170B500F014
:103A4000C9F900BF097EFC3E00F007B84FF0000046
:103A500081EA030101F00041704781EA030100F0AF
:103A600007BAF0BCBDE8004122494FF000007047A2
:103A7000FFFDFBF9F7F5F4F2F0EEEDEBE9E8E6E433
:103A8000E3E1E0DEDDDBDAD8D7D5D4D3D1D0CFCDBA
:103A9000CCCBCAC8C7C6C5C4C2C1C0BFBEBDBCBBF3
:103AA000BAB9B8B7B6B5B4B3B2B1B0AFAEADACABEE
:103AB000AAA9A8A8A7A6A5A4A3A3A2A1A09F9F9EC8
:103AC0009D9C9C9B9A99999897979695959493937A
:103AD000929191908F8F8E8E8D8C8C8B8B8A898911
:103AE0008888878786858584848383828281818094
:103AF0000000FF070000F87F51EA030C17D41CF503
:103B0000801F58BFBCF5801F00F10680994218BF86
:103B1000704708BF9042704707D711F5801F58BF04
:103B200013F5801F19D499427047894270471CF5DC
:103B3000801F08D5BCF5801FF7D58B4218BF704792
:103B400008BF824270474FF4001C1CEB410F38BF86
:103B50001CEB430F01D28B42704770B500F03AF96D
:103B6000922449004FF000514FF08053FFF75EBEA2
:103B70004FEA41034FEA5353A3F58063D3F11E0389
:103B8000C8BFD3F1210C0CDD4FF0004242EAC12244
:103B900042EA505232FA03FC8CEAE17CACEBE17071
:103BA0007047102BC4BF0020704703F5787CBCF130
:103BB000FF3F04D06FF0004282EA2100704770B5E9
:103BC00000F008F94992248000207047F2E70000D5
:103BD0004FEA1153A3F58063D3F11E03A8BFD3F1BD
:103BE000200C08DB4FF0004242EAC12252EA505258
:103BF00032FA03F0704709420BD4102BC4BF0020E7
:103C0000704703F5787CBCF1FF3F05D04FF0FF30E3
:103C100070474FF00000704770B500F0DBF800BF50
:103C20004992248000207047F0E710F0004248BF1E
:103C30004042B0FA80F310FA03F10AD0C3F11D0339
:103C400003F5806302EB03524FEA415002EBD121AE
:103C500070474FF000007047B0FA80F310FA03F19C
:103C60000AD0C3F11D0303F580634FEA03524FEA04
:103C7000415002EBD12170474FF000007047000027
:103C800070B5DFF848C11CEA111E1EBF1CEA1315EF
:103C90009EEA0C0F95EA0C0F00F06F8081EA030496
:103CA0004EEAD47EAE4421EA4C1123EA4C1341F48F
:103CB000801143F48013AEF17F7EA1FB024CA0FB88
:103CC0000365361955EB0C05A1FB034C4CF10003C1
:103CD000A0FB021C16EB0C06654153F100030942E0
:103CE00018BF46F0010613F4007F0BD14FEA0331F1
:103CF0004FEA053041EA155140EA165034036FF09F
:103D000003020AE04FEAC3214FEAC52041EA5551B8
:103D100040EA5650F4026FF0020202EB2E4201EB31
:103D2000025585EACE710AD05FEA440C18BF24F030
:103D3000004450F1000041F1000120EAD47040F24B
:103D4000FE7C624500D270BDA84214BF4FF0804493
:103D50004FF04044002E08BF0024BEF1806FA8BF82
:103D6000A1F1C041BDE8704080F2828001F1C04104
:103D700001F000414FF0000070470CEA13159EEA75
:103D80000C0F18BF95EA0C0F06D081EA030E4FF016
:103D900000000EF0004170BD00F01CF88900013EEB
:103DA00000F007B800F009B84FEA430C5FEA5C5C2A
:103DB00008D081EA030100F05BB84FEA410C5FEAEA
:103DC0005C5CF6D102494FF0000070470000FF072D
:103DD0000000F87F0EF1020E2EF0030E5EF8046B69
:103DE000364205D4012A43EB030515F5001F12D80E
:103DF000012841EB010C1CF5001F0CD80ED14FEA35
:103E0000D17C0CEB4C0C0CF1020C15F5001F08BF1B
:103E10004CEBD37C04E04FF0080C01E04FEAD37C7C
:103E20000CEB4C0526FA05F606F00706B6F1040C75
:103E300006D20EEB860CBDE870404CF0010C6047DA
:103E4000DFE80CF0090B02024FF00041A1F5002160
:103E50004FF0000070BD19461046012851EB0104D7
:103E600018BFD4F5001484BF002001F0004170BDDC
:103E70000808A0F500114FEA3101704710B591EA2A
:103E8000030F81F000413FF529AC83F0004300F0BF
:103E900009B8000010B591EA030F48BF83F0004352
:103EA0003FF51CAC841A71EB030C07D28CF0004C6C
:103EB000121943EB0C03001B61EB0C014FEA115488
:103EC000A4EB135CDFF8A4E11EEA430F18BF9EEADF
:103ED000445F00F0B48021EA045123EA6E035242A9
:103EE000C3EB6E0338BF5B1EDCF1200E25D322FA34
:103EF0000CFE10EB0E0043FA0CFE41EB0E01CCF170
:103F0000200E03FA0EFE10EB0E00CCF1200E51F144
:103F1000000129D401EB045112FA0EF2BDE8104061
:103F200058BF7047401C1CBFB2F1004F70470028BB
:103F30000CBF491C20F00100704712EB020E43EB4E
:103F4000030218BF4FF0010E4EEA4202ACF1200C02
:103F5000DCF11E0E56D943FA0CFE10EB0E00CCF12C
:103F60001E0E51F1FF31D5D50EF1010E12FA0EFEE3
:103F7000404141EB010101EB445C5FEA5C5C10D91C
:103F800001EB045110EBDE7038BFBEF1004FBDE80D
:103F9000104018BF704700280CBF491C20F00100DA
:103FA000704734D24FEAD42C24F4006411F5001188
:103FB0001BD0B1FA81F20B3AA41AA41ED2F120034D
:103FC000914030FA03F31943904001EBCC7101EBBF
:103FD0000451002CBDE81040A8BF704701F1C0415A
:103FE00001F000414FF000007047B0FA80F310FA82
:103FF00003F102D1BDE810407047E41A173C4805B0
:10400000C90AE2E701EB0451BDE8104070474910CE
:104010004FEA300001EB0451BDE8104002E04FF0E0
:10402000000170474A0008BF0042F8D0B2F5001FF7
:1040300028BF704701F000414FF0000070479EEA32
:10404000445F07D011EA5E0FBDE8104004BF0021B5
:1040500000207047BDE8104070B5FFF7BBFE00BF01
:1040600040DFF63E104683F0004170470000E0FF5D
:1040700043004FEAD30C4FEA3C0C43401FBF4007BC
:104080000CF1605113F0FE4F70471CF0006F03D12C
:104090000CF00041002070470CF0004343EA5070E0
:1040A00040EACC0010B500F001F900BF000000921A
:1040B0004FEA0001FFF7DCBE4FF00041A1F50021FF
:1040C0004FF00000704710B500F034F80CBF01202D
:1040D000002010BD10B500F02DF814BF0120002005
:1040E00010BD10B500F07AF88CBF0120002010BD83
:1040F00010B500F073F82CBF0120002010BD10B5E2
:1041000000F0A0F894BF0120002010BD10B500F011
:1041100099F834BF0120002010BD401058BFC0F1F5
:104120004040491058BFC1F140418142EFF3008047
:104130007047000050EA010C00F113801CF5000FDD
:1041400058BFBCF5000F01D48842704707D710F55F
:10415000000F58BF11F5000F15D4884270478942EF
:1041600070471CF5000F04D5BCF5000FF7D5814250
:1041700070474FF0807C1CEB400F38BF1CEB410FA9
:1041800001D28142704710B500F090F892244900A6
:104190004FF000504FF08051FFF7BFBFC10DD1F17C
:1041A0009E0206DB4FEA002343F0004323FA02F0AD
:1041B0007047004207D54FEA4001B1F1FE4F02D2ED
:1041C0004FF00000704710B500F070F8499224805D
:1041D000002070476FEA20007047000050EA010C91
:1041E00000F113801CF5000F58BFBCF5000F01D47F
:1041F0008842704707D710F5000F58BF11F5000F20
:1042000015D488427047894270471CF5000F04D5C9
:10421000BCF5000FF7D5814270474FF0807C1CEB56
:10422000400F38BF1CEB410F01D28142704710B5DF
:1042300000F03CF8922449004FF080504FF00051BC
:10424000FFF76BBF50EA010C00F113801CF5000F63
:1042500058BFBCF5000F01D48842704707D710F54E
:10426000000F58BF11F5000F15D4884270478942DE
:1042700070471CF5000F04D5BCF5000FF7D581423F
:1042800070474FF0807C1CEB400F38BF1CEB410F98
:1042900001D28142704710B500F008F8922449001D
:1042A0004FF000504FF08051FFF737BF0EF1020E74
:1042B0002EF0030E5EF8044B244204D44FEA410270
:1042C000B2F17F4F11D84FEA4003B3F17F4F0CD8C2
:1042D0000ED14FEAD07C0CEB4C0C0CF1020CB2F17D
:1042E0007F4F08BF4CEBD17C04E04FF0080C01E09D
:1042F0004FEAD17C0CEB4C0324FA03F404F00704DE
:10430000B4F1040C06D20EEB840CBDE810404CF066
:10431000010C6047DFE80CF0070802024FF0004094
:10432000A0F5800010BD0846420018BFD2F180728F
:1043300088BF00F0004010BDFF2141EAD050C00509
:1043400070470CF00F03092B08BF082000F05980BC
:104350000A2B0BD0082B18BF704708BF1CF0400F6A
:104360000AD04FF000004FF0000170471CF0400FE2
:1043700018BF4FF0004070471CF0100F08D000F03D
:104380007F4220F0704342EAD3014FEA4370704706
:1043900000F0604021F07F4242EA000201F07F40DD
:1043A00040EA727070474FF0FF0C4CF4E06C1CEA6E
:1043B00011531CBF9CEA030C9445C2BFDA4201EBC7
:1043C00002517047002B0DD0BCF1000F0FD001F04F
:1043D0000041002AA4BF41F0E04141F07F614FF06D
:1043E0000000704701F000414FF00000704750EAB4
:1043F00001334FF09B0C18BF4CF0806C7FF40EAA79
:1044000070471CF4801F11D01CF4E02F03D06FEA1A
:10441000CC31490070474FF04050EFF3008222F05A
:10442000704242EA000282F3008870474FF00000B9
:1044300070470000000000004FBB610567ACDD3F26
:10444000182D4454FB21E93F9BF681D20B73EF3FBB
:10445000182D4454FB21F93FE2652F227F2B7A3C33
:10446000075C143326A6813CBDCBF07A8807703CEC
:10447000075C143326A6913CC4EB98999999C9BF5F
:10448000711623FEC671BCBF6D9A74AFF2B0B3BF94
:104490009AFDDE522DDEADBF2F6C6A2C44B4A2BF54
:1044A0000D5555555555D53FFF8300922449C23FC0
:1044B0006E204CC5CD45B73F513DD0A0660DB13FF4
:1044C000EB0D76244B7BA93F11DA22E33AAD903F06
:1044D0004C5555555555A53F7751C1166CC156BF22
:1044E0009015CB19A001FA3EAD529C804F7E92BE32
:1044F000C4B1B4BD9EEE213ED43888BEE9FAA8BD51
:10450000000000000000000000004054FB21F93FC3
:104510003163621A61B4D03D0000601A61B4D03DCD
:104520007370032E8A19A33B0000002E8A19A33B47
:10453000C14920259A837B3900000000000000005B
:104540006E83F9A22915444ED15727FCC0DD34F5FE
:10455000999562DB4190433CAB6351FE61C5BBDE84
:104560003A6E24B7E0D24D42EA2E49061C92D10998
:104570001CEB1DFE3EA729B1F53582E88444BB2E15
:1045800026709CE9417E5FB439D69139F439538362
:104590008B5F849C3B28F9BDFF97F81F0F9805DEC1
:1045A0008B112FEF1F6D0A5ACF7E366DB709CB27BF
:1045B000663F464F2DEA5F9EC7BA27757BF1E5EB54
:1045C000F739073DEA92528AB15FFB6B085D8D1F98
:1045D0004630035600000000A6F810111111813F6B
:1045E000D561C119A0012ABF7DFEB157E31DC73EA9
:1045F000EB9C2B8AE6E55ABE7CD5CF5A3AD9E53DED
:104600000000000000000000010203040607080982
:104610000000000001020304010202030405060772
:1046200008090A0B0C0D0E0F101000005046000870
:10463000000000201000000028010008604600086B
:1046400010000020280800004401000800000000BD
:10465000010000001000000000127A0000000000BD
:04000005080000ED02
:00000001FF
